:020000040800F2
:10000000D0200020050100089D2D0008512800087F
:10001000ED2B0008330C0008C1350008000000007B
:10002000000000000000000000000000192E000881
:10003000DD0D000800000000A12D00081B2E0008A7
:100040001F0100081F0100081F0100081F01000810
:100050001F0100081F0100081F0100081F01000800
:100060001F0100081F0100081F0100081F010008F0
:100070001F0100081F0100081F0100081F010008E0
:100080001F0100081F0100081F0100081F010008D0
:100090001F0100081F0100081F0100081F010008C0
:1000A0001F0100081F0100081F0100081F010008B0
:1000B000912E00081F0100081F0100081F01000801
:1000C0001F0100081F0100081F0100081F01000890
:1000D0001F01000891350008A1350008B13500085E
:1000E0001F0100081F0100081F010008DFF810D0E1
:1000F00000F076FB00480047C5400008AFF30080E1
:10010000D02000200648804706480047FEE7FEE76B
:10011000FEE7FEE7FEE7FEE7FEE7FEE7FEE7FEE7B7
:100120008D2E0008ED000008202A04DB203A21FA79
:1001300002F00021704721FA02F3D040C2F1200200
:100140009140084319467047004870470C4E00081C
:1001500010B50446FFF7F8FF0068005D00F00100ED
:1001600010BD40EA01039B0703D009E008C9121F34
:1001700008C0042AFAD203E011F8013B00F8013B61
:10018000521EF9D27047D2B201E000F8012B491E8D
:10019000FBD270470022F6E710B513460A46044624
:1001A0001946FFF7F0FF204610BD421C10F8011B56
:1001B0000029FBD1801A704730B505460020034660
:1001C00000E05B1C934205D2EC5CC85C201A01D1B4
:1001D000002CF6D130BD00000FB400B58DB010A9D1
:1001E00009900B9000914FF0FF300A9000200C9086
:1001F00005480690054807906A4609A80F9900F03F
:1002000009F90DB05DF814FB310400084F04000833
:100210002DE9FF5F1D464FF0FF3BD5E901469146B2
:100220005F464FF00008A9697F1C01988847296A3A
:10023000824688470028F6D1BAF1FF3F0CD024F45B
:10024000C064002E19DD600614D5BAF12B0F09D059
:10025000BAF12D0F0ED103E0584604B0BDE8F09F6F
:1002600044F48064A9697F1C01988847761E824601
:10027000002E02DDBAF1300F03D0B9F1000F26D005
:1002800032E0A969761E44F400747F1C0198884707
:100290008246002E05DDBAF1780F06D0BAF1580F6C
:1002A00003D0B9F1000F10D01EE0B9F1000F02D059
:1002B000B9F1100F18D1A969761E24F400747F1CBF
:1002C000019888478246102002E0082000E00A20BA
:1002D000814609E008FB0908A969761E44F4007408
:1002E0007F1C019888478246002E05DD494650460E
:1002F00000F07BF80028EDDAE96901988847A0054D
:1003000002D46FF00100A8E7E00725D1600613D5FD
:10031000600502D5C8F1000000E0404629680A1DCA
:100320002A600968220501D5087015E0220701D569
:10033000088011E008600FE02868011D296000684E
:10034000210502D580F8008006E0210702D5A0F83B
:10035000008001E0C0F8008038467EE730B50B46EB
:10036000014600202022012409E021FA02F59D42E5
:1003700005D303FA02F5491B04FA02F52844151EB9
:10038000A2F10102F1DC30BD2DE9F05F054600204D
:1003900092469B4688460646814640241BE02846F6
:1003A000414647462246FFF7BFFE53465A46C01A0B
:1003B000914110D311461846224600F023FA2D1A17
:1003C00067EB01084F4622460120002100F01AFA8F
:1003D00017EB00094E41201EA4F10104DFDC484662
:1003E00031462A464346BDE8F09F3A2800D23038CD
:1003F00020F02002412A01D3A2F13700884201D324
:100400004FF0FF307047000002681144137801601C
:1004100018467047D16004495161044911620021B6
:100420001161114600F010BA0904000851010008DA
:10043000426842B1016811F8013B23B1521EC0E984
:100440000012184670470121C160881E704742683B
:100450005AB1C368016843B983688B4205D0491E0D
:10046000521CC0E90012002070474FF0FF30704767
:100470002DE9FE4F804681EA0300C00F0C46009034
:1004800021F0004123F00045B8EB0200A94105D25C
:100490004046214690461C460B46024623F000404B
:1004A000104347D0270DC7F30A00C3F30A51029047
:1004B000401A019040286BDAC3F3130040F4801B0C
:1004C0000098924620B10023D2EB030A63EB0B0B9A
:1004D00001985946C0F14002504600F093F9064693
:1004E0000D4650465946019A00F09BF910EB080062
:1004F0006141002487EA115284EAE7731A4340D02D
:10050000009A62B3019A012A4FEA075215DC001BD8
:1005100061EB02014FF0004202EA0752CDE90042CE
:10052000001C41F5801132462B4600F034FB03B02D
:10053000BDE8F08F40462146F9E7001B61EB020160
:10054000001C41F5801300185B412018A2F500172C
:1005500047EB030140EAD570B6196D4111E06D0813
:100560004FEA360645EAC0754FEA0752001B61EBB9
:100570000201001C41F5801149084FEA30000019C2
:10058000514132462B4603B0BDE8F04F00F0F4BABB
:100590000098012240000023D0EB020263EBE073DD
:1005A000009821464FEAE074B8EB000061EB0401CB
:1005B000E9E783F000435BE781F0004158E72DE96C
:1005C000FE4F81EA030404F0004421F0004100944E
:1005D0004FF0000B23F0004350EA01045ED052EAD2
:1005E00003045BD0C3F30A54C1F30A552C44A4F2AC
:1005F000F3340194A0FB0254C1F3130141F48011C0
:10060000C3F3130343F4801301FB024400FB034EC6
:10061000840A970A44EA815447EA8357A4FB07688F
:1006200002958D0A05FB07854FEA932C04FB0C54B9
:100630002705029D4FEA065847EA1637B5EB08052D
:100640006EEB070C870E920E47EA811742EA83127F
:10065000A7FB0201B6EB0B0164EB00042B0D43EA90
:100660000C335E1844EB1C50DA465146E7FB02019E
:10067000C5F313044FEA0B3343EA14534FEA043231
:10068000019C43EA0603A4F10C040294009CCDE90A
:1006900000B400F080FA03B0BDE8F08F00200146FE
:1006A000F9E72DE9F04D81EA030404F0004B21F055
:1006B000004514464FF0000A23F0004150EA0502BD
:1006C00020D054EA01021DD0C5F30A570246C5F3F3
:1006D0001303C1F31300C1F30A5640F4801543F429
:1006E0008013A7EB0608101BD64608F2FD3873EB03
:1006F000050002D308F1010801E092185B41B8F14E
:10070000000F03DA00200146BDE8F08D00204FF411
:100710008011064684460EE0171B73EB050705D3D0
:10072000121B63EB050306434CEA010C49084FEA30
:10073000300092185B4150EA0107EDD152EA030004
:1007400012D082EA040083EA0501084305D0101B99
:10075000AB4106D20122002306E000224FF0004305
:1007600002E06FF0010253101AEB06004CEB085147
:1007700010EB0A0041EB0B01BDE8F04D00F0FCB9B5
:10078000C1F30A52C1F3130140F2FF3341F4801167
:100790009A4202DA00200146704740F233439A42FF
:1007A000A2F2334202DC5242FFF7BEBC00F02AB88C
:1007B00030B5041E71F1000404DB4FF000444042E8
:1007C00064EB0101141E73F1000405DB1C464FF0BD
:1007D0000043524263EB0403994208BF904230BD8C
:1007E000064C074D06E0E06840F0010394E807007E
:1007F00098471034AC42F6D3FFF77CFC9C4E0008BF
:10080000BC4E0008202A04DB203A00FA02F1002046
:1008100070479140C2F1200320FA03F3194390403E
:100820007047202A06DBCB17203A41FA02F043EA50
:10083000E07306E041FA02F3D040C2F12002914099
:1008400008431946704700002DE9F34F8BB04FF075
:10085000000801F10C000C464FF0010B46460DF16B
:10086000080A01906269012101989047051E2DD068
:10087000252D2CD0216A8847C0B1626901210198D9
:100880009047216A88470028F7D1411E6269019884
:10089000904700E0761CA1690B988847216A884739
:1008A0000028F7D1E1690B988847DBE7A1690B982D
:1008B00088470746A84201D1761CD3E7E1690B9827
:1008C00088477F1C02D1B8F1000F6FD047E10027A5
:1008D00062693D463946019890472A2804D16269E9
:1008E0000121019890470125DFF888926269012172
:1008F00001989047A0F130010A290AD24F45E5DC62
:1009000007EB870100EB4107303FDFD445F01005CE
:10091000ECE7E90601D46FF000476C280AD04C28B8
:1009200014D0682815D06A280DD074281CD07A28D5
:100930001AD01DE062690121019890476C2802D00D
:1009400045F0040514E045F002050DE045F02005F2
:100950000AE06269012101989047682802D045F0B9
:10096000080505E045F4006562690121019890479A
:10097000C4E9015765283DD019DC58287AD00CDC31
:10098000452837D004DC252826D0412831D131E054
:1009900046282FD047282CD12CE05B2877D061281F
:1009A00028D063287CD0642823D15AE0D1E06F2876
:1009B00048D008DC66281DD067281BD0692821D0C4
:1009C0006E2816D127E0702845D0732868D0752886
:1009D00047D078280DD14DE0A1690B98884705468E
:1009E00025283FF469AFE1690B9888476D1C3FF4F7
:1009F0006AAFB4E023466A466FF001000B99AFF38B
:100A000000809FE045F040006060A80723464FF05B
:100A1000000236D43EE0E8077FF447AF2068011DAE
:100A200021600068290501D506701BE7290701D55B
:100A3000068017E7A90703D5F117C0E9006111E7A0
:100A400006600FE745F040006060A80723464FF0BE
:100A5000080216D41EE040F60E0125EA010060608F
:100A600016E045F040006060A80723464FF00A02F8
:100A700007D40FE045F040006060A80708D5234682
:100A800010226FF001000B99AFF300805AE007E0ED
:100A9000234610226FF001000B99FFF7B9FB51E0DC
:100AA0004FF000094F464B46632802D05B2807D021
:100AB00041E02079C00601D40120A06001273AE07E
:100AC00062690121019890475E2805D14FF0010924
:100AD0006269494601989047216939B900210A465F
:100AE000534643F82120491C0829FADBB0B3216999
:100AF00069B9C11700EBD16253110AEB830122F0EF
:100B00001F02821A01200B68904003430B60626948
:100B10000121019890475D28E8D1B9F1000F09D073
:100B20000020514651F82020D24341F82020401C9B
:100B30000828F7DB02AB224600976FF001000B9903
:100B4000AFF3008000280CDA401C08D1BBF1000F85
:100B500005D04FF0FF300DB0BDE8F08FFFE7404605
:100B6000F9E7E90701D108F1010806444FF0000B4D
:100B700078E60000CCCCCC0C10B5141E73F1000448
:100B800008DA401C41F1000192185B411A4301D17F
:100B900020F0010010BD2DE9F04D92469B4611B1A9
:100BA000B1FA81F202E0B0FA80F220329046FFF70B
:100BB00029FE04460F4640EA0A0041EA0B0153466B
:100BC0005A46084313D0114653EA010019D0C8F120
:100BD00040025046FFF7A8FA05460E4650465946D1
:100BE0004246FFF70FFE084305D0012004E02046EF
:100BF0003946BDE8F08D0020054346EAE0762C43F7
:100C000037430A986305E40AA0EB08000022FD0AB6
:100C100044EA47540A3002D500200146E9E70105BD
:100C200010196941DDE9084500196941BDE8F04D39
:100C3000A2E700BFFEE7000010B560210348FFF700
:100C4000A9FA00200149087010BD00004C0A0020DC
:100C500001490860704700001800002010B500200E
:100C600018E0144901EB001108700021114A02EB51
:100C7000001251600F4A02EB001291600D4A02EB24
:100C8000001211730C4A22F810100C4A42F820107E
:100C9000411CC8B20328E4DB002009490860094967
:100CA0000860094908600120084908700848FFF7F2
:100CB000CFFF10BDB80C002082000020680E00207D
:100CC00074000020780000207C00002080000020BC
:100CD000613F000810B500200349087003F0B0F927
:100CE00002A002F0F5F910BD880000205B4C4F47D0
:100CF0005D204465627567206C6F6720737973743B
:100D0000656D20696E697469616C697A65640D0A44
:100D1000000000000FB470B5C2B005460E4625486D
:100D20000078854203DA42B070BC5DF814FB3046AF
:100D300003F0A2F900B9F6E700240EB1304600E056
:100D40001DA01F4A009052F82530C4F5807102AAF8
:100D500010191CA202F046FC0444FF2C0DDA49A82D
:100D60000190C4F5807102AA1019019B489A02F003
:100D700053FC04440020019000BF002C0CDDFF2C2C
:100D80000ADC0D222046641C02A90A54FF2C03DC55
:100D90000A222046641C0A54002C08DDA1B202A8D5
:100DA00002F03CF9A2B202A9022001F05FFF00BFED
:100DB000B9E70000880000204D41494E00000000C6
:100DC000184D00085B25735D5B25735D20000000F6
:100DD000014908707047000088000020704772B613
:100DE00000BFFEE70146002291F82100022808D04A
:100DF0000420886300BF002081F8200000BF01208C
:100E000070470868006820F00E000B6818600868DA
:100E1000006820F001000B68186091F84030012054
:100E20009840CB6B5860012081F8210000BF002062
:100E300081F8200000BF1046E2E7000070B50446CC
:100E4000002594F82100022803D00420A063012586
:100E500048E02068006820F00E00216808602068E3
:100E6000006820F00100216808601F49206888425E
:100E700001D1012026E01C4914312068884201D1AB
:100E800010201FE0184928312068884201D18015C0
:100E900018E015493C312068884201D1801411E0E6
:100EA000114950312068884202D14FF4803009E066
:100EB0000D4964312068884202D14FF4801001E06E
:100EC0004FF08070084908394860012084F82100FB
:100ED00000BF002084F8200000BF606B10B12046E6
:100EE000616B8847284670BD0800024070B5044613
:100EF00000F0AEF906462546681C10B1044800789B
:100F0000054400BF00F0A4F9801BA842FAD370BDCD
:100F1000940000202DE9F8470346002294466EE134
:100F20004FF0010808FA02F4D1F8008008EA040042
:100F3000A0427DD1DFF8DCA2D1F80480A8EB0A0939
:100F4000D0453AD014DCB8F1030F50D009DCB8F129
:100F5000000F31D0B8F1010F1CD0B8F1020F49D108
:100F600020E0B8F1110F18D0B8F1120F42D11EE0F5
:100F7000B9F5881F25D006DCB9F5803F20D0B9F53A
:100F8000801F37D11AE0B9F5001F18D0B9F5041F3A
:100F900030D117E0D1F80CC02DE0D1F80C8008F169
:100FA000040C28E0D1F80C8008F1080C23E0D1F8FB
:100FB0000C8008F10C0C1EE000BF00BF00BF00BF9A
:100FC00000BF00BFD1F80880B8F1000F02D14FF088
:100FD000040C0BE0D1F80880B8F1010F03D14FF0F9
:100FE000080C1C6102E04FF0080C5C6103E04FF05C
:100FF000000C00E000BF00BFFF2801D8984601E0C8
:1010000003F104084646FF2802D84FEA820803E0AD
:10101000A2F108084FEA88084746D6F800804FF04A
:101020000F0909FA07F928EA09080CFA07F900E09C
:1010300088E048EA0908C6F80080D1F8048008F082
:101040008058B8F1805F7DD100BFDFF8CC81D8F83F
:10105000188048F00108DFF8C091C9F81880C84628
:10106000D8F8188008F00108CDF8008000BF00BF54
:101070004FEAB9384FEA920958F829504FEA827876
:101080004FEA18794FF00F0808FA09F825EA080521
:10109000DFF88881434502D14FF0000816E0DFF801
:1010A0008081434502D14FF001080FE0DFF87481E1
:1010B000434502D14FF0020808E0DFF86C81434558
:1010C00002D14FF0030801E04FF004084FEA8279A3
:1010D0004FEA197908FA09F848EA0505DFF84C8162
:1010E0004FEA920948F82950D1F8048008F4801892
:1010F000B8F5801F0AD1DFF83881D8F8008048EAB7
:101100000008DFF82C91C9F8008009E0DFF82081A1
:10111000D8F8008028EA0008DFF81491C9F80080A8
:10112000D1F8048008F40018B8F5001F10D1DFF8DA
:10113000008108F10408D8F8008048EA0008DFF8C8
:10114000F09000E05AE009F10409C9F800800DE0D0
:10115000DFF8DC8008F10408D8F8008028EA0008ED
:10116000DFF8CC9009F10409C9F80080D1F80480B7
:1011700008F40038B8F5003F0ED1DFF8B480A8F1CC
:101180000408D8F8008048EA0008DFF8A490A9F124
:101190000409C9F800800DE0DFF89480A8F1040884
:1011A000D8F8008028EA0008DFF88490A9F1040943
:1011B000C9F80080D1F8048008F48038B8F5803F81
:1011C0000ED1DFF86C80A8F10808D8F8008048EA52
:1011D0000008DFF85C90A9F10809C9F800800DE06B
:1011E000DFF84C80A8F10808D8F8008028EA000849
:1011F000DFF83C90A9F10809C9F80080521CD1F829
:10120000008028FA02F8B8F1000F7FF489AEBDE83B
:10121000F887000000001110001002400008014093
:10122000000C014000100140001401400800014082
:1012300008040140024693680B400BB1012000E016
:10124000002070470AB1016101E00B04036170479F
:1012500001480068704700008C00002003480068C7
:101260000349097808440149086070478C00002050
:101270009400002010B50848006840F010000649AE
:101280000860032000F0A8F80F2000F007F800F035
:101290002BF8002010BD00000020024070B504466D
:1012A0000E4800784FF47A71B1FBF0F00C490968F0
:1012B000B1FBF0F5284600F09DFC08B1012070BD9F
:1012C000102C07D200222146501E00F047F8054896
:1012D000046001E00120F2E70020F0E79400002024
:1012E000980000209000002008B500BF11488069D8
:1012F00040F001000F4988610846806900F0010054
:10130000009000BF00BF00BF0846C06940F0805099
:10131000C8610846C06900F08050009000BF00BF5F
:1013200000BF0549486820F0E06040F00070486068
:1013300000BF08BD00100240000001400146084601
:10134000002809DB00F01F0301229A4043099B009B
:1013500003F1E023C3F8002100BF70472DE9F05FDF
:1013600080460D461646002702F070F907463946BA
:101370002A46334601F00700C0F1070ABAF1040F0C
:1013800002D94FF0040A01E0C0F1070AD14600F18A
:10139000040ABAF1070F02D24FF0000A01E0A0F1EF
:1013A000030AD4464FF0010A0AFA09FAAAF1010A1F
:1013B0000AEA020A0AFA0CFA4FF0010B0BFA0CFBCC
:1013C000ABF1010B0BEA030B4AEA0B042146404642
:1013D00002F044F9BDE8F09F00BF00F00702064BA1
:1013E00019684FF6FF031940044B0B4343EA0221EF
:1013F000014B196000BF70470CED00E00000FA05DA
:1014000070B504460D460CB9012070BD5A480068FD
:1014100000F00700A8420ED25748006820F00700ED
:101420002843554908600846006800F00700A842B4
:1014300001D00120E9E7207800F0020002281DD148
:10144000207800F00400042805D14C48406840F49E
:10145000E0604A494860207800F00800082805D17B
:101460004648406840F460504449486043484068FA
:1014700020F0F000A168084340494860207800F05F
:10148000010078B36068012806D13C48006800F488
:10149000003090B90120B8E76068022806D13748CB
:1014A000006800F0007040B90120AEE733480068E2
:1014B00000F0020008B90120A7E73048406820F09A
:1014C0000300616808432D494860FFF7C1FE0646E6
:1014D00009E0FFF7BDFE801B41F28831884202D946
:1014E000032092E707E02548406800F00C0061689F
:1014F000B0EB810FEDD12048006800F00700A84252
:101500000ED91D48006820F0070028431A490860DA
:101510000846006800F00700A84201D0012074E7E7
:10152000207800F00400042807D11448406820F413
:10153000E060E168084311494860207800F0080045
:10154000082808D10D48406820F46050216940EA1D
:10155000C1000A49486000F03FF808494968C1F3F2
:101560000311074A515CC8400649086006480068F4
:10157000FFF794FE002048E70020024000100240E0
:10158000524D00089800002090000020014800689B
:10159000704700009800002000B5FFF7F7FF0449EE
:1015A0004968C1F30221034A515CC84000BD0000F4
:1015B00000100240624D000800B5FFF7E7FF044944
:1015C0004968C1F3C221034A515CC84000BD000014
:1015D00000100240624D000870B500210022002476
:1015E00000230020134D696801F00C05F5B1042DAE
:1015F00002D0082D19D101E00F4819E00F4DC1F3B9
:101600008346AB5D01F4803555B10A4D6D68C5F375
:1016100040450B4E725D084D5D43B5FBF2F402E0B0
:10162000084D03FB05F4204602E000BF024800BF5E
:1016300000BF70BD0010024000127A00404D00084B
:10164000504D000800093D00F8B504460CB90120D2
:10165000F8BD207800F00100002878D0F8484068F4
:1016600000F00C0004280CD0F548406800F00C0095
:10167000082811D1F248406800F48030B0F5803F6E
:101680000AD1EF48006800F4003000285FD060689D
:1016900000285CD10120DBE700BF6068B0F5803F27
:1016A00006D1E748006840F48030E549086028E04A
:1016B000606858B9E248006820F48030E04908606A
:1016C0000846006820F4802008601AE06068B0F5E1
:1016D000A02F0BD1DA48006840F48020D849086078
:1016E0000846006840F4803008600AE0D44800688A
:1016F00020F48030D24908600846006820F4802039
:10170000086000BF606888B1FFF7A2FD054606E0EB
:10171000FFF79EFD401B642801D9032098E7C848C5
:10172000006800F400300028F2D010E0FFF790FDD0
:10173000054606E0FFF78CFD401B642801D9032015
:1017400086E7BF48006800F400300028F2D1207816
:1017500000F00200022857D1B948406800F00C00A0
:1017600050B1B748406800F00C00082818D1B448C0
:10177000406800F4803098B9B148006800F0020079
:1017800020B12069012801D0012061E7AC48006840
:1017900020F0F800616940EAC100A949086033E01F
:1017A0002069E8B10120A7490860FFF751FD05460F
:1017B00006E0FFF74DFD401B022801D9032047E753
:1017C0009F48006800F002000028F2D09C480068A2
:1017D00020F0F800616940EAC1009949086013E00F
:1017E000002098490860FFF733FD054606E0FFF743
:1017F0002FFD401B022801D9032029E790480068EB
:1018000000F002000028F2D1207800F0080008283B
:101810002DD1A069B8B101208B490860FFF718FDF0
:10182000054606E0FFF714FD401B022801D90320FE
:101830000EE78348406A00F002000028F2D0012041
:1018400001F0B0FA13E000207F490860FFF700FDC7
:10185000054606E0FFF7FCFC401B022801D90320E7
:10186000F6E67748406A00F002000028F2D12078BE
:1018700000F00400042873D100277148C06900F00B
:10188000805070B900BF6E48C06940F080506C490C
:10189000C8610846C06900F08050009000BF00BFDA
:1018A00001276A48006800F48070B0B96748006892
:1018B00040F4807065490860FFF7CAFC054606E001
:1018C000FFF7C6FC401B642801D90320C0E65F482F
:1018D000006800F480700028F2D000BFE0680128A2
:1018E00006D15748006A40F001005549086227E0D8
:1018F000E06858B95248006A20F001005049086277
:101900000846006A20F00400086219E0E068052833
:101910000BD14B48006A40F0040049490862084670
:10192000006A40F0010008620AE04548006A20F0C1
:101930000100434908620846006A20F0040008627A
:1019400000BFE068A0B1FFF783FC054609E0FFF7A0
:101950007FFC401B41F28831884202D9032077E6A0
:1019600022E03748006A00F002000028EFD012E0C1
:10197000FFF76EFC054608E0FFF76AFC401B41F2EA
:101980008831884201D9032062E62D48006A00F0C0
:1019900002000028F0D1012F05D12948C06920F0AC
:1019A00080502749C86100BFE069C8B32448406837
:1019B00000F00C00082860D0E069022848D100201F
:1019C00020490866FFF744FC054606E0FFF740FCA7
:1019D000401B022801D903203AE61948006800F0AC
:1019E00000700028F2D1206AB0F5803F07D114487A
:1019F000406820F40030A168084311494860D4E9E8
:101A0000080108430E49496821F4741108430C4940
:101A1000486001200B490866FFF71AFC054607E0FD
:101A20003DE0FFF715FC401B022801D903200FE61B
:101A30000348006800F000700028F2D02FE000009A
:101A40000010024000004242800442420070004008
:101A5000002014490866FFF7FBFB054606E0FFF788
:101A6000F7FB401B022801D90320F1E50E4800686E
:101A700000F000700028F2D111E0E069012800D1E7
:101A8000E6E50948466806F48031206A814204D1BF
:101A900006F47011606A814201D00120D8E500206F
:101AA000D6E50000000042420010024010B5044696
:101AB0000CB9012010BD606A38B96068B0F5827F4A
:101AC00000D105E00021E16102E0002121616161B6
:101AD0000021A16294F8510028B9002084F8500038
:101AE000204600F043F8022084F851002068006886
:101AF00020F0400021680860A08800F482702189ED
:101B000001F404410843A18901F400610843217CE8
:101B100001F002010843217D01F001010843218BFE
:101B200001F400710843217F01F0380108432021AE
:101B3000095D01F080010843218D01F40051084343
:101B4000216808600421A06901EA1040216848600A
:101B50002068C06920F400602168C86100206065C9
:101B6000012084F851000020A4E7000010B586B0E1
:101B70000446002002900390049005901A492068C2
:101B800088422FD100BF1948C06940F480401749EE
:101B9000C8610846C06900F48040019000BF00BFE2
:101BA00000BF0846806940F00800886108468069E7
:101BB00000F00800019000BF00BF4FF420400290E9
:101BC000022003900320059002A90948FFF7A2F91B
:101BD0004FF48040029000200390049002A9044832
:101BE000FFF798F906B010BD003800400010024021
:101BF000000C014070B504462546681EB0F1807F98
:101C000001D301200FE0681E4FF0E02148610F2151
:101C10004FF0FF3001F022FD00204FF0E0218861FD
:101C200007200861002070BD7047704730B502463C
:101C30000B4600BF92F83C00012801D1022030BDC4
:101C4000012082F83C0000BF022082F83D001068AD
:101C500044681068816824F07004186804431068B0
:101C60004460104D1068A8420BD01068B0F1804F4E
:101C700007D00D4D1068A84203D00C4D1068A84243
:101C800005D121F08001586801431068816001206E
:101C900082F83D0000BF002082F83C0000BF00BF7A
:101CA000CDE70000002C0140000400400008004087
:101CB00010B504460CB9012010BD94F83D0028B9B8
:101CC000002084F83C00204600F026F8022084F82A
:101CD0003D00211D206801F0E3F8012084F8460052
:101CE00000BF84F83E0001213F20015540200155EE
:101CF0004120015500BF00BF012084F8420043206D
:101D00000155442001554520015500BF012084F8AC
:101D10003D000020D0E7000038B504462068B0F14F
:101D2000804F15D100BF0B48C06940F00100094940
:101D3000C8610846C06900F00100009000BF00BF04
:101D4000002211461C20FFF709FB1C20FFF7F6FAC2
:101D500038BD000000100240014691F83D00012806
:101D600001D001207047022081F83D000868C0685A
:101D700040F001000B68D860124B086898420BD005
:101D80000868B0F1804F07D00F4B0868984203D025
:101D90000E4B086898420CD10868806800F0070272
:101DA000062A0CD00868006840F001000B68186033
:101DB00005E00868006840F001000B68186000202A
:101DC000D0E70000002C0140000400400008004063
:101DD0002DE9F04104460D46002700BF94F83C0071
:101DE000012802D10220BDE8F081012084F83C00E6
:101DF00000BF022084F83D002068866826F0770640
:101E000026F47F46206886602868502833D00CDC92
:101E1000202850D004DC00284BD0102851D149E0B4
:101E2000302849D040284CD139E060282DD0702886
:101E300007D0B0F5805F03D0B0F5005F41D10DE071
:101E400041E0D5E902136A68206801F063F8206870
:101E5000866846F077062068866034E0D5E902138C
:101E60006A68206801F056F82068806840F4804075
:101E70002168886027E0EA686968206801F05EF8F8
:101E80005021206801F051F81DE0EA686968206877
:101E900001F067F86021206801F047F813E0EA6874
:101EA0006968206801F04AF84021206801F03DF897
:101EB00009E000BF00BF00BF2968206801F035F8C5
:101EC00001E0012700BF00BF012084F83D0000BFF2
:101ED000002084F83C0000BF384684E7704710B506
:101EE000044620680069C0F34000D8B12068C0688B
:101EF000C0F34000B0B16FF002002168086101201A
:101F000020772068806900F0030018B12046FFF7B1
:101F1000E5FF05E0204600F0ADF8204600F0ABF804
:101F20000020207720680069C0F38000D8B12068C5
:101F3000C068C0F38000B0B16FF004002168086190
:101F4000022020772068806900F4407018B1204694
:101F5000FFF7C4FF05E0204600F08CF8204600F0B3
:101F60008AF80020207720680069C0F3C000D8B14B
:101F70002068C068C0F3C000B0B16FF008002168ED
:101F80000861042020772068C06900F0030018B1C0
:101F90002046FFF7A3FF05E0204600F06BF820463F
:101FA00000F069F80020207720680069C0F3001075
:101FB000D8B12068C068C0F30010B0B16FF0100055
:101FC00021680861082020772068C06900F440700B
:101FD00018B12046FFF782FF05E0204600F04AF8DE
:101FE000204600F048F8002020772068006900F0C3
:101FF000010058B12068C06800F0010030B16FF0F6
:10200000010021680861204600F036F82068006968
:10201000C0F3C01058B12068C068C0F3C01030B120
:102020006FF08000216808612046FFF7FDFD206801
:102030000069C0F3801058B12068C068C0F38010F8
:1020400030B16FF0400021680861204600F01DF8B3
:1020500020680069C0F3401058B12068C068C0F320
:10206000401030B16FF02000216808612046FFF772
:10207000DCFD10BD7047704710B504462068B0F114
:10208000804F01D102F02CFE10BD70477047000058
:1020900038B5044600BF002000902068006800901A
:1020A00020684068009000BF00BF00BF0020009083
:1020B00020680068009020684068009000BF00BF62
:1020C00000BF0020009020680068009020684068F1
:1020D000009000BF00BF0F492068884205D101224F
:1020E0000D490E4800F09EFA12E00D492068884222
:1020F00005D101220B490C4800F094FA08E00B4985
:102100002068884204D1012209490A4800F08AFA6D
:1021100038BD000000380140BC00002074090020D8
:102120000048004005000020040A00200044004050
:1021300004000020BC0900202DE9F84F0446206867
:1021400005682068C668206847694FF00009CA46DC
:1021500005F00F09B9F1000F0AD105F0200038B1E0
:1021600006F0200020B1204601F07CF8BDE8F88F91
:10217000B9F1000F7BD007F0010018B906F4907098
:10218000002874D005F0010030B106F4807018B159
:10219000606C40F00100606405F0040030B107F0AD
:1021A000010018B1606C40F00200606405F00200AC
:1021B00030B107F0010018B1606C40F004006064B9
:1021C00005F0080048B106F0200010B907F0010042
:1021D00018B1606C40F008006064606C002845D065
:1021E00005F0200028B106F0200010B1204601F0D3
:1021F00039F820684069C0F3801A606C00F008006C
:1022000010B9BAF1000F2CD0204600F0E5FF20688D
:10221000406900F0400000B300BF00BF21681431E6
:1022200051E8001F21F040002168143141E800020C
:10223000002AF3D100BFE06B50B17748E16B4863EF
:10224000E06BFEF7FBFD88B1E06B416B88470DE06A
:102250002046FFF71DFF09E009E02046FFF718FFC1
:1022600004E02046FFF714FF002060647EE7206B47
:10227000012877D105F01000002873D006F0100077
:102280000028FAD000BF002000902068006800906D
:1022900020684068009000BF00BF2068406900F0DF
:1022A000400000285FD0E06B006840681FFA80F8AB
:1022B000B8F1000F55D0A08D404552DDA4F82E8016
:1022C000E06B8069202843D000BF00BF21680C313B
:1022D00051E8001F21F4807021680C3141E80002B0
:1022E000002AF3D100BF00BF00BF2168143151E8BC
:1022F000001F21F001002168143141E80002002A8A
:10230000F3D100BF00BF00BF2168143151E8001FA6
:1023100021F040002168143141E80002002AF3D185
:1023200000BF202084F842000020206300BF00BFCF
:1023300021680C3151E8001F21F0100021680C3198
:1023400041E80002002AF3D100BFE06BFEF74AFD2E
:1023500002206063A08DE28D801A81B22046FFF7D3
:1023600095FE03E742E0A08DE18D401A1FFA80F848
:10237000E08DD0B3B8F1000F37D000BF00BF2168A7
:102380000C3151E8001F21F4907021680C3141E8B4
:102390000002002AF3D100BF00BF00BF2168143142
:1023A00051E8001F21F001002168143141E80002CA
:1023B000002AF3D100BF202084F8420000202063CF
:1023C00000BF00BF21680C3151E8001F21F0100050
:1023D00021680C3141E80002002AF3D100BF02203D
:1023E000606341462046FFF751FEBFE605F08000DE
:1023F00030B106F0800018B1204601F04FF8B5E684
:1024000005F0400030B106F0400018B1204600F061
:1024100019FFABE600BFA9E6C531000810B50446B8
:102420000CB9012010BDA06900B100E000BF94F814
:10243000410028B9002084F84000204600F02AF826
:10244000242084F841002068C06820F400502168EE
:10245000C860204600F084FF2068006920F49040A6
:10246000216808612068406920F02A0021684861DD
:102470002068C06840F400502168C8600020606493
:10248000202084F8410084F842000020606300BFEF
:10249000C8E7000010B586B0044600200290039003
:1024A0000490059059492068884237D100BF5848A8
:1024B000806940F48040564988610846806900F48C
:1024C0008040019000BF00BF00BF0846806940F017
:1024D000040088610846806900F00400019000BF94
:1024E00000BF48150290022003900320059002A926
:1024F0004848FEF70FFD4FF48060029000200390E3
:10250000049002A94348FEF705FD0022114625204C
:10251000FEF724FF2520FEF711FF75E03E492068F5
:10252000884236D100BF3A48C06940F4003038498B
:10253000C8610846C06900F40030019000BF00BFC8
:1025400000BF0846806940F0040088610846806941
:1025500000F00400019000BF00BF042002900220A0
:1025600003900320059002A92A48FEF7D3FC082017
:10257000029000200390049002A92648FEF7CAFCAE
:10258000002201212620FEF7E9FE2620FEF7D6FED6
:102590003AE022492068884236D100BF1C48C06911
:1025A00040F480201A49C8610846C06900F48020C0
:1025B000019000BF00BF00BF0846806940F00800DE
:1025C00088610846806900F00800019000BF00BFE4
:1025D00008150290022003900320059002A91048DC
:1025E000FEF798FC4FF400600290002003900490E6
:1025F00002A90B48FEF78EFC002202212720FEF7DD
:10260000ADFE2720FEF79AFE06B010BD003801404F
:102610000010024000080140004400400048004013
:10262000000C014070B504460D46164694F8420071
:1026300020280BD105B10EB9012070BD0020206308
:1026400032462946204600F009FFF6E70220F4E76B
:1026500010B5044623492068884216D122480088D4
:10266000FF2808D821490A781F490888411C1E4BB9
:1026700019801F490A54FEF7EBFD1E49086001222C
:102680001A491D48FFF7CEFF2AE01C4920688842FE
:102690001DD1FEF7DDFD1A490968884211D319489A
:1026A0000088B0F5007F08D217490A7815490888D4
:1026B000411C144B198015490A54FEF7C9FD1449F1
:1026C0000860012210491348FFF7ACFF08E01249E7
:1026D0002068884204D1012210491148FFF7A2FF67
:1026E00010BD00000038014006000020BC000020A2
:1026F0001801002008000020740900200048004054
:10270000140000200C00002005000020180200200A
:1027100010000020040A00200044004004000020B3
:10272000BC0900202DE9F84F04460E46174699468D
:102730004FF0000A94F8410020284AD106B117B999
:102740000120BDE8F88F00206064212084F841005A
:10275000FEF77EFD8246A784E784A068B0F5805F1F
:1027600004D1206910B90025B04602E035464FF08B
:1027700000081BE05346002280212046CDF800903F
:1027800000F0BCFE08B10320DBE745B9B8F8000053
:10279000C0F308002168486008F1020803E02878C7
:1027A000216848606D1CE08C401EE084E08C0028AD
:1027B000E0D15346002240212046CDF8009000F0A1
:1027C0009DFE08B10320BCE7202084F841000020D2
:1027D000B7E70220B5E710B5034693F8410020287B
:1027E00013D101B10AB9012010BD19629A84DA84AB
:1027F00000205864212083F841001868C06840F028
:1028000080001C68E0600020EEE70220ECE700009A
:1028100010B504460B492068884203D1002000F01F
:1028200081FA0DE008492068884202D100F094FC4A
:1028300006E006492068884202D1022000F072FAC0
:1028400010BD000000380140004400400048004036
:1028500000BFFEE70021002009E0074A02EB00125A
:1028600092791AB1012282400A43D1B2401C042855
:10287000F3DB0846704700002000002070B50025FB
:1028800012E0114800EB0514A1882068FEF7D2FC85
:1028900008B1012000E00020A071A0792072012081
:1028A000E0710020E0606D1C042DEADB0020074988
:1028B0000860012006490870FFF7CCFF0446214656
:1028C00004A000F08BFB70BD200000206000002001
:1028D000640000205B494F5D20496E6974204F4BB6
:1028E0002C20696E697469616C20737461746573FE
:1028F0003A203078253032580D0A00002DE9F04199
:10290000FEF7A6FC07461C480068381A0A2801D2C0
:10291000BDE8F08118480760002628E0174800EB62
:102920000614A1882068FEF785FC08B1012000E0AC
:1029300000200546207AA84203D00020E0712572CD
:1029400014E0E079032803DAE079401CE0710DE03F
:10295000A079A8420AD0A571E068401CE060084850
:10296000007818B1F0B2294602F06AF8761C042EFD
:10297000D4DB00BFCCE70000600000202000002076
:102980006400002000B585B0002001900290039003
:10299000049000BF3C48806940F010003A498861CB
:1029A0000846806900F01000009000BF00BF00BF23
:1029B0000846806940F0200088610846806900F080
:1029C0002000009000BF00BF00BF0846806940F0B3
:1029D000040088610846806900F00400009000BF90
:1029E00000BF00BF0846806940F0080088610846C3
:1029F000806900F00800009000BF00BF0122802124
:102A00002248FEF71FFC012205212148FEF71AFC8F
:102A1000002241F208211E48FEF714FC00224FF468
:102A200001411A48FEF70EFC48F280100190012087
:102A30000290002003900220049001A91348FEF7A1
:102A400069FA41F20D2001900120029000200390CC
:102A50000220049001A90E48FEF75CFA02200190C2
:102A6000002002900120039001A90948FEF752FAC4
:102A7000F020019000200290039001A90448FEF785
:102A800049FA05B000BD00000010024000080140F6
:102A9000000C014010B50E480E4908604FF48270DA
:102AA000486000210B488160C160016141614FF4C1
:102AB000007181610021C1610162416281620A216C
:102AC000C162FEF7F3FF08B1FEF789F910BD0000FF
:102AD000003800401C09002000B587B0002003909A
:102AE000049005900690019002904FF080401449A8
:102AF0000860472048600021114881604FF6FF714F
:102B0000C160002101618161FFF7D2F808B1FEF7D1
:102B100066F94FF48050039003A90948FFF758F96C
:102B200008B1FEF75CF900200190029001A9044869
:102B3000FFF77CF808B1FEF752F907B000BD0000BE
:102B40008814002010B50B480B4908604FF416504C
:102B50004860002108488160C16001610C21416129
:102B600000218161C161FFF759FC08B1FEF737F917
:102B700010BD0000003801407409002010B50B485A
:102B80000B4908604FF4E13048600021084881603B
:102B9000C16001610C21416100218161C161FFF7C8
:102BA0003DFC08B1FEF71BF910BD000000440040D9
:102BB000BC09002010B50B480B4908604FF4965033
:102BC0004860002108488160C16001610C214161B9
:102BD00000218161C161FFF721FC08B1FEF7FFF818
:102BE00010BD000000480040040A002000BFFEE7BE
:102BF0000146032901DB03A07047044850F8210077
:102C0000FAE70000554E4B4E4F574E00344D00082A
:102C100070B5002520E06B206843114901EB80046A
:102C2000104850F8250020600F4850F825006060DB
:102C300004F1080001F0DDFE04F1900001F0E9FF6D
:102C4000002004F5CE7404F8020C20606060A060DF
:102C500001202073681CC5B2032DDCDB70BD0000B1
:102C6000840F0020284D0008344D00082DE9F04164
:102C700005460F469046032D03DA17B1B8F1000F51
:102C800001D1BDE8F081012D04D14146384600F064
:102C9000C5F9F6E76B2068430C4901EB800494F812
:102CA000A80100B9EDE74246394604F1900001F071
:102CB000BBFF0646002E07DDD4F8A0013044C4F85F
:102CC000A001284601F068FF00BFDAE7840F00206A
:102CD00070B505460C4604B970BD2046FDF765FA8F
:102CE00086B2324621462846FFF7C0FF00BFF3E711
:102CF00070B5002411E06B206043094901EB8005A9
:102D000095F8A80100B906E0012C00D103E02046A7
:102D100001F042FF00BF601CC4B2032CEBDB70BDAE
:102D2000840F0020F8B50546032D00DBF8BD012D0A
:102D300002D100F011FAF9E76B206843164901EB64
:102D4000800606F19004002772B6002084F8060180
:102D5000B4F80401002816DDB4F80201205C0090EC
:102D600004F581742188481CC11700EB1161091218
:102D7000A0EB012121806088401E6080012020712D
:102D8000A4F58174012762B627B101226946306833
:102D9000FFF721FD00BFC9E7840F002000BFFEE759
:102DA0007047000008B508490968C9084FF47A72ED
:102DB000B1FBF2F14143009100BF00BF00994A1EF0
:102DC00000920029F9D108BD9800002010B500221A
:102DD0004FF400410548FEF735FA00200449087019
:102DE0000449086004A000F0F9F810BD0008014093
:102DF0006C000020700000205B52454C41595D2062
:102E0000496E6974204F4B2C2073746174653D4F7B
:102E100046460D0A00000000704710B501F08AFE1A
:102E2000FEF71CFA10BD00B58FB0282105A8FDF7EC
:102E3000B1F914216846FDF7ADF9012005900004B1
:102E40000690002007900120099002200C90C103F9
:102E50000D914FF4E0110E9105A8FEF7F5FB08B1B6
:102E6000FDF7BDFF0F20009002200190002002908E
:102E70004FF4806003900020049002216846FEF722
:102E8000BFFA08B1FDF7ABFF0FB000BD70470000FF
:102E900010B50248FFF723F810BD00008814002089
:102EA00010B50268184B984208D0B0F1804F05D099
:102EB000164B984202D0164B984203D122F0700272
:102EC0004B681A43104B984208D0B0F1804F05D0A0
:102ED0000E4B984202D00E4B984203D122F440721E
:102EE000CB681A4322F080034C6943EA0402026073
:102EF0008B68C3620B688362034B984201D10B69F4
:102F000003630123436110BD002C01400004004015
:102F10000008004030B50C46816821F47F4142EA48
:102F2000032525432943816030BD0A46816821F08D
:102F3000700142F0070319438160704730B50B46BA
:102F40001446026A056A25F001050562816921F0CF
:102F5000F00141EA041122F00A021A43816102627F
:102F600030BD30B50B461446026A056A25F01005DF
:102F70000562816921F4704141EA043122F0A00226
:102F800042EA03128161026230BD000010B50020E8
:102F90000849A1F80002A1F80202A1F8040281F890
:102FA0000602A1F808024FF4007103A000F016F821
:102FB00010BD0000AC0A00205B55415254325D2028
:102FC000496E6974204F4B2C2062756666657220CD
:102FD00073697A653A2025640D0A00000FB410B5B4
:102FE000A2B0249818B922B010BC5DF814FB25A833
:102FF0000190802102A8019B249A00F00DFB044659
:1030000000200190002C06DB802C00DB7F24A1B285
:1030100002A800F003F800BFE5E70000F8B5044699
:103020000D4605B104B9F8BD0026002772B6002090
:103030002AE02549B1F80412B1F5007F07DB2249E7
:10304000B1F80812491C204AA2F808121EE0215CBF
:103050001D4AB2F800221C4B99541A46B2F80022BD
:10306000511CCA1701EBD2525212A1EB4222A3F813
:1030700000221946B1F80412491C1A46A2F804129B
:10308000711C8EB2411C88B2A842D2DB00BF002E58
:1030900008DD0D4890F8060220B901200A4981F8A0
:1030A0000602012762B66FB172B60748B0F8020295
:1030B0000549085C009062B6012269460348FFF7A3
:1030C0008AFB00BF00BFAEE7AC0A0020BC090020AD
:1030D00070B5044604B970BD2046FDF766F885B2A8
:1030E00029462046FFF79AFF00BFF4E738B572B6CD
:1030F000174890F8060218B91548B0F8040208B944
:1031000062B638BD1248B0F802420146B1F8021268
:10311000481CC11700EBD1514912A0EB41210C4AC8
:10312000A2F802121046B0F80402401E1146A1F89F
:103130000402012081F806020846005D009062B694
:10314000012269460348FFF746FB00BFD9E70000AC
:10315000AC0A0020BC09002038B5002572B600205A
:10316000164981F806020846B0F8040200281CDD62
:103170000846B0F80242B1F80212481CC11700EB31
:10318000D1514912A0EB41210C4AA2F8021210467B
:10319000B0F80402401E1146A1F80402012081F893
:1031A00006020846005D0090012562B625B10122A5
:1031B00069460348FFF70FFB38BD0000AC0A00204A
:1031C000BC09002070B505466C6A0020E085E084EB
:1031D0002046FEF75DFF70BD00BF00BF02680C32E5
:1031E00052E8002F22F4907102680C3242E800137A
:1031F000002BF3D100BF00BF00BF0268143252E8B9
:10320000002F22F001010268143242E80013002B63
:10321000F3D100BF016B01290ED100BF00BF0268CE
:103220000C3252E8002F22F0100102680C3242E802
:103230000013002BF3D100BF202180F842100021A1
:103240000163704710B504462068C06820F0400054
:103250002168C860202084F841002046FFF7D8FA92
:10326000002010BDF8B5044694F84200222875D11C
:10327000A068B0F5805F0CD1206950B90025A66A1E
:1032800020684068C0F308003080A06A801CA062FB
:1032900015E0A56A0026A068B0F5805F03D0A0689D
:1032A00028B9206918B920684068287004E02068AF
:1032B000406800F07F002870A06A401CA062E08D8A
:1032C000401E80B2E085002846D12068C06820F00A
:1032D00020002168C8602068C06820F480702168E0
:1032E000C8602068406920F0010021684861202002
:1032F00084F8420000206063206B012826D1002062
:10330000206300BF00BF21680C3151E8001F21F08D
:10331000100021680C3141E80002002AF3D100BFFF
:103320002068006800F0100010280AD100BF0020BB
:10333000009020680068009020684068009000BFFE
:1033400000BFA18D2046FEF7A1FE02E02046FFF758
:103350007FF90020F8BD01E00020FBE70220F9E73B
:1033600070B504462168096921F44051E2681143AF
:10337000226811612269A1681143626941EA02056C
:103380002168C96841F20C62914329432268D160E7
:103390002168496921F44071A26911432268516191
:1033A0002D4A2168914202D1FEF706F901E0FEF7AD
:1033B000F3F800EBC00101EB001162689200B1FB71
:1033C000F2F100EBC00202EB001263689B00B2FB5B
:1033D000F3F26423B2FBF3F202EBC20303EB02123B
:1033E000A1EB8201322202EB01116422B1FBF2F166
:1033F00001F0F00100EBC00202EB001263689B00D9
:10340000B2FBF3F26423B2FBF3F201EB021200EB26
:10341000C00101EB001163689B00B1FBF3F100EB0D
:10342000C00303EB00136668B600B3FBF6F3642633
:10343000B3FBF6F303EBC30606EB0313A1EB830127
:10344000322303EB01116423B1FBF3F101F00F010F
:1034500011442268916070BD0038014010B50346E8
:1034600099629A85DA8500205864222083F8420008
:10347000186928B11868C06840F480701C68E06062
:103480001868406940F001001C6860611868C068F5
:1034900040F020001C68E060002010BD014691F85B
:1034A0004100212828D18868B0F5805F0BD10869D8
:1034B00048B90A6A1088C0F308000B685860086AA7
:1034C000801C086205E00B6A581C086218780B68BB
:1034D0005860C88C401E80B2C88458B90868C0685B
:1034E00020F080000B68D8600868C06840F0400099
:1034F0000B68D860002070470220FCE72DE9F041FE
:1035000004460D4617469846069E34E0701C88B364
:103510002EB1FDF79DFEA0EB0800B0422BD900BFF5
:1035200000BF21680C3151E8001F21F4D0702168E0
:103530000C3141E80002002AF3D100BF00BF00BFF8
:103540002168143151E8001F21F001002168143175
:1035500041E80002002AF3D100BF202084F8410096
:1035600084F8420000BF002084F8400000BF032020
:10357000BDE8F081FFE7206800682840A84201D13B
:10358000012000E00020B842C0D00020F0E7000099
:1035900010B50248FEF7D0FD10BD000074090020F0
:1035A00010B50248FEF7C8FD10BD0000BC090020A0
:1035B00010B50248FEF7C0FD10BD0000040A00204F
:1035C00000BFFEE70FB4054B10B503A9044A0298EB
:1035D00000F02AF910BC5DF814FB0000D53F00088C
:1035E000D00000200FB47CB50C0009AD01D0611EE5
:1035F00000E00021CDE90001064B6A462946089803
:1036000000F012F9002C02D0009A002111707CBC4D
:103610005DF814FB2F3F00087CB50C001D461646D4
:10362000014601D0601E00E00020CDE90010064BED
:103630006A462946304600F0F7F8002C02D0009A7E
:10364000002111707CBD00002F3F00080248006877
:10365000C0F30220704700000CED00E010B5002818
:1036600004DB0A07130E054A135406E00A07140E7A
:10367000034A00F00F031B1FD45410BD00E400E008
:1036800018ED00E002E008C8121F08C1002AFAD1B4
:1036900070477047002001E001C1121F002AFBD1D2
:1036A000704700002DE9FF5F82B00021DDE90430A2
:1036B000020DDDF840B0034318D044F61050A2F2DA
:1036C000FF3242431514119801281FD0A5EB0B00BF
:1036D000401C5FEA000A4FF000064E4FDFF83891B9
:1036E000B046504615D5CAF1000413E011980124E4
:1036F0004AA3012801D16FEA0B010298119AC0E98F
:103700000031C0E9024206B0BDE8F09FCBF10000F5
:10371000DFE704460021404A491842EB0450CDE956
:10372000001012E0E00707D032463B4640464946CB
:10373000FCF745FF8046894632463B46104619460F
:10374000FCF73DFF06460F466410002CEAD1DDE988
:103750000401DDE90023BAF1000F06DAFCF72FFFC0
:1037600042464B46FCF72BFF05E0FCF79AFF42462A
:103770004B46FCF796FF04460E460022284BFDF709
:1037800017F803D84FF0FF30014607E00022254B21
:1037900020463146FCF76CFEFCF7F2FF102409E0EE
:1037A000002C0ADB0A220023FCF7EEFD039B3032DB
:1037B0001A55641E50EA0102F2D1641C039AC4F146
:1037C00011031444119A012A03D0012208430DD198
:1037D0000AE0084304D000204FF0110B119072E76B
:1037E000A3EB0B056D1E0DE05B4504DD4FF0000201
:1037F00005F1010504E003DA4FF00002A5F101052F
:10380000002AECD002981199C0E90231C0E90045C4
:1038100079E70000000014400000F03F3000000095
:103820000000F0430000E03F2DE9FF4F95B09A46BD
:10383000884606460025EEE1252877D10024274654
:10384000F94A0121039400E0044316F8013F203BAC
:1038500001FA03F01042F7D130782A2811D06FF026
:103860002F033078A0F13002092A16D8039A44F0C9
:10387000020402EB820203EB42021044761C039026
:10388000EFE758F8042B0392002A03DA504244F47D
:103890000054039044F00204761C30782E2816D190
:1038A00016F8010F44F004042A280DD06FF02F02FF
:1038B0003078A0F13003092B09D807EB870302EB1E
:1038C0004303C718761CF3E758F8047B761C30785E
:1038D0006C280FD006DC4C2817D068280DD06A2839
:1038E00014D104E0742810D07A280FD10DE044F4EC
:1038F00000140AE044F4801401E044F440147278A7
:10390000824202D104F58014761C761C3078662839
:103910000BD013DC582877D009DC002875D0452857
:10392000F6D04628F4D047281AD193E118E063284E
:1039300035D0642879D0652812D18BE1702873D0F6
:1039400008DC6728F1D069286FD06E280DD06F2869
:1039500006D1ACE073282CD0752874D0782853D0C9
:103960005246179990476D1C54E1C4F30250022847
:1039700009D003280DD0D8F8001004280DD00D6010
:1039800008F1040846E1D8F80010EA17C1E900522E
:10399000F6E7D8F800100D80F2E70D70F0E718F8A0
:1039A000041B8DF8001000208DF80100EB4601206B
:1039B00003E058F804BB4FF0FF3061074FF00001FF
:1039C00002D40DE009F101018946B9420FDA8145BF
:1039D000F8DB1BF809100029F4D108E009F1010116
:1039E00089468142FADB1BF809100029F6D10398B9
:1039F0005346A0EB090721463846179A00F080FA93
:103A0000284400EB090507E044E008E10DE01BF85D
:103A1000010B524617999047B9F10109F7D2534665
:103A200021463846179AF2E039E00A21C4F30252DF
:103A30004FF0000B0091022A06D058F8040BC11772
:103A4000032A09D00AE023E008F1070020F007026A
:103A5000F2E80201904605E000B2C117042A01D144
:103A600040B2C117002906DA0A460021404261EB44
:103A700002012D2202E0220504D52B228DF804201C
:103A8000012203E0E20701D02022F7E7914657E048
:103A90000A2100E010214FF0000B00910BE01021F3
:103AA0004FF0000B44F004040827009103E00820C5
:103AB0004FF0000B0090C4F30252022A05D058F8D0
:103AC000040B0021032A08D008E008F1070020F0C9
:103AD0000702F2E80201904603E080B2042A00D116
:103AE000C0B24FF0000922072AD53278702A07D0D9
:103AF000DDF800C08CF0100C5CEA0B0C05D00EE079
:103B000040228DF80420012208E050EA010306D08B
:103B100030238DF804308DF8052002229146009B59
:103B200083F0080353EA0B030AD150EA010201D1E2
:103B3000620705D530228DF804204FF001097F1E61
:103B40003278582A04D039A20C920CAA02920BE0C7
:103B50003BA2F9E75B46009AFCF716FC0C9B9B5CCA
:103B6000029A521E0292137050EA0102F2D1029898
:103B700004A9081A00F1200B600702D524F4803450
:103B800000E001275F4502DDA7EB0B0000E000200D
:103B900000EB0B01009003984944401A0390E003A6
:103BA00006D453462146179A039800F0A9F9054414
:103BB000002706E001A85246C05D179990476D1C8A
:103BC0007F1C4F45F6DBE0030CD553462146179A80
:103BD000039800F095F9054404E030205246179907
:103BE00090476D1C0099481E00900029F5DC08E004
:103BF0000298029952460078491C02911799904701
:103C00006D1CBBF10001ABF1010BF1DC5BE100F0DD
:103C100065F90544761C307800287FF40DAE19B0A4
:103C20002846BDE8F08F000009280100303132330A
:103C300034353637383961626364656600000000E8
:103C400030313233343536373839414243444546D2
:103C500000000000600700D4062708F1070020F0EC
:103C60000700F0E80223804603F0004C5FEA0C00F6
:103C700001D097A009E0200501D596A005E0E00756
:103C800001D095A001E0AFF24C001390307823F002
:103C9000004365280CD006DC452809D046281DD0F5
:103CA00047287FD13BE0662818D067287AD136E0D4
:103CB0000021112F01DB112000E0781CCDE900016B
:103CC00004A90CA8FFF7EEFCDDE90D010C9A4FF0FA
:103CD000000B07F10109109200914EE04FF00040F7
:103CE0000097CDE9011004A90CA8FFF7DBFCDDE982
:103CF0000D020C9B0F994FF0000B91461093009210
:103D000011B9791C00EB0109B7EB090003D4C0F12C
:103D1000FF3B07F10109A9EB0700019042E0012FE9
:103D200000DA01270021112F01DD112000E03846C3
:103D3000CDE9000104A90CA8FFF7B4FCDDE90D01F1
:103D40000C9A00914FF0000BB946109221070FD446
:103D5000009A4A4503DA914601E0A9F10109B9F157
:103D6000010F05DD109AA9F10101515C3029F4D051
:103D7000B84202DA10F1040F03DA0121CDE9011093
:103D800010E0002803DC8344A9EB000102E0411CA1
:103D9000494500DD8946A0EB0B00401C01904FF027
:103DA00000400290200705D40198484502DB4FF0FF
:103DB000FF30019000208DF84B0002980DF14B0769
:103DC000B0F1004F25D002200C902B200D900298CE
:103DD00000280CDA404202902D200D9007E00A21C5
:103DE0000298FCF7BBFA3031029007F8011D0C99DC
:103DF000481E0C900029F2DC02980028EFD1791EB1
:103E00000D980870307800F0200040F0450007F869
:103E1000020D11A8C01BC01D02901398007800B1BC
:103E2000012000EB0901019801EBE07102980144C7
:103E30000398401A401E0390E00306D453462146DF
:103E4000179A039800F05CF805441398007818B1AD
:103E50005246179990476D1CE00323D553462146DF
:103E6000179A039800F04CF805441BE0BBF1000FD3
:103E700007DB0098584504DD1098179910F80B00DF
:103E800001E0179930205246904701980BF1010B41
:103E9000401E05F10105019004D12E2052461799CC
:103EA00090476D1CB9F10001A9F10109DEDC05E0C4
:103EB00017F8010B5246179990476D1C0299481E3E
:103EC00002900029F4DC53462146179A03989EE697
:103ED0002D0000002B000000200000002DE9F04123
:103EE000044600251E461746880404D405E03946DA
:103EF0002020B0476D1C641EF9D52846BDE8F0812E
:103F00002DE9F041044600251E469046C80301D520
:103F1000302700E02027880404D505E041463846D4
:103F2000B0476D1C641EF9D52846BDE8F0814A688B
:103F3000002A06D00A68531C0B6010704868401EA7
:103F40004860704710B502460023002003E0145C6F
:103F50006340441CE0B28842F9DB184610BD000003
:103F6000F8B505460C461448006878B12046FCF7C1
:103F70001CF986B23246214628460F4B1B689847EB
:103F80000E480068401C0D49086008E0214628469C
:103F9000FEF79EFE09480068401C08490860284654
:103FA000FEF726FE0646334605A208A1012000942E
:103FB000FCF7B0FEF8BD0000740000207C0000207B
:103FC00054585B25735D3A2025730000524F5554B9
:103FD0004552000013B50C4601216846FFF71EF854
:103FE000012269460220FEF741FE00981CBD000038
:103FF00010B5002208210248FDF724F910BD000089
:10400000000C014010B5012208210248FDF71AF901
:1040100010BD0000000C014010B500224FF40071EB
:104020000148FDF70FF910BD000C014010B5012249
:1040300051020248FDF706F910BD0000000C0140D6
:104040000B48007800B17047002009E0002100EB28
:104050000012084B995400EB00121A441174401CD2
:104060001028F3DB01200249087000BFEBE70000D5
:1040700089000020740E002070B505460DB1287827
:1040800008B9012070BDFFF7DBFF002414E004EB4A
:1040900004100B49085C70B104EB0411084A88183D
:1040A0000F222946FCF788F828B904EB04100449CC
:1040B0000844007CE6E7641C102CE8DB0120E1E703
:1040C000740E0020FDF7D6F8FEF7ADFEFEF75AFCA1
:1040D000FEF738FDFEF7DEFCFEF750FDFEF76AFD49
:1040E000FEF7FAFC5F48FDF737FEFEF74FFFFEF7DD
:1040F000C5FBFCF7A1FDFEF769FEFEF789FDFCF7A5
:10410000ADFDFCF7E7FD0120FCF762FE56A0FFF7CE
:1041100059FA5448FDF720FE01225C495C48FEF73D
:1041200081FA01225B495C48FEF77CFA002000F02E
:1041300047FA012259495A48FEF774FA002000F064
:10414000A3FB4FF47A710A2000F0CAFB002000F0B4
:1041500067FA00F0B5FA53A0FFF734FA5DA0FFF755
:1041600031FA654800686549B0FBF1F4214664A066
:10417000FFF728FA68A0FFF725FA00F0C7FB00F068
:10418000AFFA6EE0FEF7B2FFFEF7B2FDFEF7B6FB48
:104190006C48008800283BDDFDF75AF86A49096839
:1041A000401A142834D972B66648048822466749F2
:1041B0006748FBF7D6FF00206249088062B6022CF0
:1041C0001BDB63480078AA2817D161484678A01EF7
:1041D00085B25F4FBF1C2A4631465E48FFF7F2F9B1
:1041E000002D09DD2A4639460220FEF73FFD2A460A
:1041F00039460120FEF73AFD09E0224654490220E3
:10420000FEF734FD224652490120FEF72FFD00BF84
:1042100051480088002824DDFDF71AF84F49096845
:10422000401A14281DD972B64B48048822464C49BE
:104230004C48FBF796FF00204749088062B6AA2049
:104240004949087001204870224646494648801C6A
:10425000FBF787FFA01C82B243490020FEF706FD52
:1042600000BF8FE7881400200D0A5B444542554784
:104270005D20312E20E590AFE58AA82054494D32CB
:1042800020E4B8ADE696AD0D0A0000000400002061
:10429000BC09002005000020040A0020BC0000200A
:1042A000740900200D0A3D3D3D3D3D3D3D3D3D3DF8
:1042B0003D3D3D3D3D3D3D3D3D3D3D3D3D3D3D3D2E
:1042C0003D3D3D3D3D3D3D3D3D3D3D3D3D3D0D0A81
:1042D000000000004533322D3433335442482D530F
:1042E00043204170706C69636174696F6E20537410
:1042F00061727465640D0A009800002040420F004E
:1043000053797374656D20436C6F636B3A20256439
:10431000204D487A0D0A00003D3D3D3D3D3D3D3D6F
:104320003D3D3D3D3D3D3D3D3D3D3D3D3D3D3D3DBD
:104330003D3D3D3D3D3D3D3D3D3D3D3D3D3D3D3DAD
:104340000D0A0000060000200800002018010020CF
:1043500018040020104E00080C000020100000205F
:10436000180200201805002018070020002003492B
:10437000086003490860034908607047B0000020E6
:10438000B4000020B8000020014611B96FF002000F
:1043900070470248006808800020F9E7B800002054
:1043A00030B503460C460BB104B112B96FF00200F0
:1043B00030BD1448006818B900201080401EF7E78F
:1043C00000201080002115E00F48104D2D68405D41
:1043D00058540E480068401CC0F309000B4D28607B
:1043E00008480068401E074D28601088401C108057
:1043F000481C81B2A14203DA024800680028E3D1D8
:104400000020D5E7B8000020D0180020B40000201C
:104410000748006850B106480068401E044908601B
:104420000846006810B90120024908707047000072
:10443000C0000020C400002010B502210D48FCF788
:10444000F9FEA0B9FCF704FF044607E0FCF700FF03
:10445000001B642802D36FF0010010BD0221054843
:10446000FCF7E8FE0028F1D00220FCF73FFD002019
:10447000F3E70000000C01400548007810B94FF048
:10448000FF30704700200249087000BFF9E70000C4
:10449000AC00002010B5FFF769FF10BD10B5044651
:1044A0002046FFF771FF10BD70B504460D46164655
:1044B000324629462046FFF773FF70BD0848007852
:1044C00010B14FF0FF3070470020064908600649E0
:1044D0000860064908600120014908700020F2E7E1
:1044E000AC000020B0000020B4000020B800002084
:1044F00070B50546FFF7A0FF04460CB1204670BD1D
:1045000035B1012D0FD0022D18D0032D2CD120E074
:10451000002280211C48FCF795FE002201211B4847
:10452000FCF790FE23E0012280211748FCF78AFE69
:10453000002201211548FCF785FE18E000228021A9
:104540001148FCF77FFE012211461048FCF77AFE65
:104550000DE0012280210C48FCF774FE0122114677
:104560000A48FCF76FFE02E06FF00200C7E700BFE9
:104570000520FCF7BBFCFFF75FFF04460CB12046AB
:10458000BDE70020BBE7000000080140000C01402F
:1045900070B504460D4604B115B96FF0020070BD48
:1045A0004FF6FF732A4621460448FEF7BBF806463D
:1045B00016B16FF00100F2E70020F0E77409002067
:1045C00070B505461348007810B14FF0FF3070BD4C
:1045D000FFF774FF044614B14FF0FF30F7E735B929
:1045E0000D480E490A6802600979017104E00A4821
:1045F0002968016029790171074800F0F1F8044643
:104600001CB1FFF739FF2046E1E70120014908709E
:104610000020DCE79C0000209D0000206A4D00087F
:1046200070B5054615B94FF0FF3070BD28210F4811
:10463000FBF7B0FD00200D49087081F82500084601
:1046400029680162297980F82410203000F0C8F828
:1046500004460CB12046E8E7002000F0EDF80446DF
:104660000CB12046E1E70020DFE70000D400002085
:104670002DE9F04104460D4616461F4614B10DB112
:1046800006B11FB94FF0FF30BDE8F0810A2D02DA04
:104690004FF0FF30F8E72078542802D1607858288E
:1046A00002D04FF0FF30EFE73B46324602A1E01C5C
:1046B000FBF792FD0020E7E725642E25642E00001D
:1046C00010B500F05DF804460CB1204610BD012085
:1046D0000249087081F825000020F7E7D400002087
:1046E00010B594B0254890F8250008B914B010BD55
:1046F0002248007820B1012806D0022836D134E0C3
:1047000001201E49087035E00020039003A904A889
:1047100000F0BAFA40B3002002900190039881B2F1
:1047200001AB02AA04A8FFF7A3FF0446DCB91348B3
:104730004068401C114948600298886101984861AE
:104740000846C0690199884202D20C490198C861A3
:1047500000F058F9012000F043F93220FCF7C6FBC5
:10476000002000F03DF900BF04E003E0022003490F
:10477000087000BF00BF00BFB8E70000D4000020F1
:1047800010B50C48007810B96FF0050010BD0A484C
:10479000007810B16FF00100F8E7FFF77BFE0446E8
:1047A00014B14FF0FF30F1E70120034908700020F9
:1047B000ECE700009C000020A200002010B5044699
:1047C000C0200649087008462168C0F80110217908
:1047D00041710621FFF7DCFE10BD0000D01400205F
:1047E00070B5054615B96FF0030070BDFFF724FEE4
:1047F000044614B16FF00200F7E70320FFF778FEDC
:10480000044614B16FF00200EFE72846FFF7D6FF29
:104810006420FCF76BFB0020FFF76AFE044614B12E
:104820006FF00200E1E7034829680160297901710E
:104830000020DAE79D00002070B504462046FFF70F
:1048400057FE054615B16FF0020070BD0020FCE771
:1048500070B505460E4605B116B96FF0030070BD80
:104860000848007810B96FF00500F8E7314628468F
:10487000FFF78EFE044614B16FF00200EFE7002050
:10488000EDE700009C00002070B505461C21124891
:10489000FBF780FC002010490870487635B90846BF
:1048A0000E490A6842610979017604E00A482968DC
:1048B00041612979017608481430FFF791FF0446D9
:1048C0000CB1204670BD0020FFF7B6FF04460CB1C6
:1048D0002046F7E70020F5E7FC0000206A4D0008BD
:1048E000024602B111B94FF0FF30704706488260AE
:1048F0000020054B58601846C160002018611870F0
:10490000012058760020F0E7FC00002070B588B048
:104910003248407E08B908B070BDFCF799FC0446E7
:104920002E48007830B1012808D0022842D0032850
:104930004CD14AE00120294908704BE027484068E3
:1049400026498968884206D303202449087000203C
:1049500000F056F93EE021480069201A1F49C96855
:10496000884226D31D484068431C1C482021826889
:10497000684600F0EDF80546002D16DD294668462C
:10498000FFF766FF06467EB914484068401C13498D
:10499000486008460461012000F032F93220FCF73B
:1049A000A5FA002000F02CF900BF02200B49087086
:1049B00000BF0FE009480069201A0849C968884209
:1049C00002D301200549087004E003E003200349F5
:1049D000087000BF00BF00BF9DE70000FC00002082
:1049E00010B5044614B1FFF70DFB01E0FFF700FB23
:1049F00010BD002120F8801F41808180C180803857
:104A0000704700000D48C069B8B10C48C0690B4937
:104A10004968411A0948C160C06958B10748C0686F
:104A2000642148430549C969B0FBF1F0C1B20348AC
:104A3000017402E00021014801747047D400002095
:104A40002DE9F0419AB004460D460220631C23A2D2
:104A50002021CDE9005012A8FEF7C4FD0646701EC5
:104A6000C1B20DF14900FFF76DFA8046C6F1200191
:104A700012AA901943461EA2FEF7B4FD0DB11EA066
:104A800000E01FA00246611C1EA0FEF7A7FAAA20A4
:104A90008DF8080001208DF8090012A8FBF785FBAE
:104AA00087B23A4612A90DF10A00FBF75AFBB81C6F
:104AB00082B202A90020FEF7D9F812A916A0FEF7CB
:104AC0008DFA1B48006828B112AA29462046184BC7
:104AD0001B6898471AB0BDE8F08100002444495F84
:104AE0004556454E542C25642C25642C25642A00FB
:104AF000253032580D0A00004849474800000000A0
:104B00004C4F57005B494F5D2043482564202D3EA4
:104B10002025730D0A0000005B494F5D205246348A
:104B200033332054583A20222573220D0A00000006
:104B30006800002010B500F0CFF80448006820B1EC
:104B400002480068401E0149086010BD00000020B6
:104B50002DE9F84305460E46174698460DB1102E2E
:104B600002DA0020BDE8F8833B4607A2314628461A
:104B7000CDF80080FEF736FD0446002C01DDA0B222
:104B8000F0E70020EEE7000054582E2530336C7516
:104B90002E2530336C752E00F8B505466B20684322
:104BA000164901EB800606F19004002772B694F8CE
:104BB0000601D0B9B4F80401002816DDB4F80201EA
:104BC000205C009004F581742188481CC11700EB1B
:104BD00011610912A0EB012121806088401E6080D4
:104BE00001202071A4F58174012762B627B101224A
:104BF00069463068FDF7EFFDF8BD0000840F002026
:104C000010B5044614B1FFF711FA01E0FFF704FAFA
:104C100010BD002100F5807001804180818081718C
:104C20000181A0F58070704770B503460C460025E1
:104C300072B6002021E0B3F80411FF2905DDB3F8B6
:104C40000811491CA3F8081119E0215CB3F80061B0
:104C50009955B3F80061711CCE1701EB1666361238
:104C6000A1EB0626A3F80061B3F80411491CA3F8D0
:104C70000411691C8DB2411C88B29042DBDB00BF7D
:104C800062B6284670BD0000F8B506460D4606B16E
:104C90000DB90020F8BD0F48007808B90020F9E7E9
:104CA0006846FFF7FBFB04460CB10020F2E7BDF8B5
:104CB000000008B90020EDE72A46FF213046FFF743
:104CC000F3FB04460CB10020E4E700200149087022
:104CD0000120DFE7C400002000B5FFF799FB00BD0D
:104CE00010B50B480068401C094908600948046871
:104CF0000BE0A068401CA060D4E90110884203D3F7
:104D00000020A06020688047E468002CF1D110BD2D
:104D1000CC000020C8000020744E00086C4E000833
:104D2000644E00087C4E000874090020BC09002075
:104D3000040A0020844E00088C4E0008944E00089F
:104D400002030405060708090A0B0C0D0E0F1010CC
:104D50000102000000000000000001020304060739
:104D60000809000000000102030400001A1707C12F
:104D7000C1C141542B444556545950453D3F004113
:104D8000542B4657434F44453D3F00004040404070
:104D9000404040404041414141414040404040400E
:104DA00040404040404040404040404005020202F8
:104DB000020202020202020202020202202020205B
:104DC0002020202020200202020202020290909065
:104DD0009090901010101010101010101010101053
:104DE00010101010101010020202020202888888AF
:104DF00088888808080808080808080808080808B3
:104E00000808080808080802020202408C4D000841
:104E10000D0A5B44454255475D20E694B6E588B0EF
:104E2000E69DA5E887AA20E8AEBEE5A4875B2564D9
:104E30005D20E79A84E6B688E681AF2C20E69C895F
:104E4000E69588E695B0E68DAEE995BFE5BAA63A57
:104E500020256420E5AD97E88A82EFBC815C720A68
:104E6000000000005741524E20000000494E464FBE
:104E70002000000044454255470000004552524F73
:104E80005200000055415254310000005541525427
:104E9000320000005541525433000000BC4E00085F
:104EA00000000020D400000084360008904F000865
:104EB000D4000020FC1F0000943600080000000011
:104EC00000000000000000000000000000000000E2
:104ED000000000000000000000000000000C014085
:104EE000100000000000000000000000000C014065
:104EF000200000000000000000000000000C014045
:104F0000400000000000000000000000000C014014
:104F10008000000000000000000000000000000011
:104F20000100000000000000000000000000000080
:104F30000000000000000000000000000100000070
:104F40000000000000000000000000001000000051
:104F5000010000000024F400000000000000000038
:104F60000000000000000000000000000000000041
:104F70000000000000000000000000000000000031
:104F80000000000000000000000000000000000021
:04000005080000ED02
:00000001FF
